:1000000009C021C020C01FC01EC01DC01CC01BC015
:1000100085C019C011241FBECFE9CDBF10E0A0E6F6
:10002000B0E0E6EFF3E002C005900D92AA36B1070A
:10003000D9F720E0AAE6B0E001C01D92A337B207CD
:10004000E1F7A3D0D6C1DCCF18BAF89411BC85B7BC
:10005000877E806185BF85B7806285BF889508955A
:1000600018BA90E0FC01EB59FF4F208127BBFC013F
:10007000EF59FF4F808186BF90E09595879589BDA8
:100080008AE083BFCB010197F1F713BE17BA8DE168
:1000900088BB0895CF93C0E068EA71E68C2FE0DF5B
:1000A000CF5FC430C9F7CF910895CF93C3E068EA1A
:1000B00071E68C2FD5DFC150D0F76091710080912F
:1000C0007000861788F4609580E090E085D160919B
:1000D0006D0081E090E080D160916C0082E090E062
:1000E0007BD1D8DFD7DFD6DFCF91AECF80916E0046
:1000F00090916F0065E078E019D1875E994C9093FC
:100100006F0080936E008927982F92959F708927A2
:10011000982F969596958927837008951F920F9230
:100120000FB60F9211242F938F939F9380916A00A3
:1001300090916B00019690936B0080936A00809180
:100140006000882389F08091600081508093600076
:1001500022B780916C0090916D00880F991F8227C3
:1001600090936D0080936C009F918F912F910F90D1
:100170000FBE0F901F90189580916C0090916D00AC
:1001800090936F0080936E0008958DE188BB379A3D
:10019000369A3699FECF84B190E090936D008093AB
:1001A0006C0016B880E481BD789481E083BF8091B3
:1001B00060008111FCCF81E28FBD80E090E005D12D
:1001C00080958093700096B39D71953161F030F405
:1001D0009D3011F58FEF809371001EC0993151F061
:1001E0009C3151F019C06FEF80E090E0F5D0109293
:1001F000700012C08093710081E090E0E6D0C82FBB
:1002000082E090E0E2D02C2F30E0322F2227282B02
:1002100030936D0020936C0090E8C92E96E7D92E9C
:1002200097E0E92EF12C05E0C0E1D7E2A5DF10E070
:10023000209171002117A8F030E0285F3F4F032E76
:10024000000C440B550BC701B60181D0205D3E4E1A
:10025000C9010197F1F74ADF68EC7FEA01DF1F5F10
:10026000E7CF10926B0010926A000093720084DF57
:10027000B12C809171008B1530F120917200E5E670
:10028000F0E010E086B391918D71892361F4809143
:100290006A0090916B00029740F5121326C01092ED
:1002A0006B0010926A001F5F143061F710E08091BC
:1002B0006A0090916B00813A9F4008F0C5DE1123DF
:1002C000E1F2B394D6CFE0E0F0E03197F1F78E3F62
:1002D00048F48F5F80937100DDDE88EC9FEA019720
:1002E000F1F7A4CFD7DEE1DEA1CF68EC7FEA812F62
:1002F000B7DEFCDE982E181789F083E0A82ECE0119
:100300000197F1F760E27EE4892DAADEAA94A1109C
:10031000F6CF80E090E00197F1F7C7DE10926B0016
:1003200010926A001093720011E0C1CF002455278B
:1003300004C0080E591F880F991F009729F0769561
:100340006795B8F37105B9F7802D952F0895052E9F
:1003500097FB16F400940FD057FD05D014D007FC7E
:1003600002D046F408C050954095309521953F4FF6
:100370004F4F5F4F089590958095709561957F4F91
:100380008F4F9F4F0895A1E21A2EAA1BBB1BFD01A0
:100390000DC0AA1FBB1FEE1FFF1FA217B307E40764
:1003A000F50720F0A21BB30BE40BF50B661F771FBC
:1003B000881F991F1A9469F760957095809590959C
:1003C0009B01AC01BD01CF010895E199FECF8EBB29
:1003D000E09A99278DB30895262FE199FECF1CBA94
:1003E0008EBB2DBB0FB6F894E29AE19A0FBE019630
:0603F0000895F894FFCF10
:0A03F60008EFB38F770A0603120028
:00000001FF
